:1000000020080010A5010000000000000000000012
:1000100011030000110300001103000000000000A4
:1000200000000000000000000000000011030000BC
:100030001103000000000000110300001103000084
:100040001103000011030000110300001103000060
:100050001103000011030000110300001103000050
:100060001103000011030000110300001103000040
:100070001103000011030000110300001103000030
:100080001103000011030000110300001103000020
:100090001103000011030000110300001103000010
:1000A0001103000011030000110300001103000000
:1000B00011030000110300001103000011030000F0
:1000C000110300002DE9F04186B000F0EBF92F4A52
:1000D0004FF41641106800F0A3FA2D48022103885E
:1000E0002C4F2D4D2D4C0491ADF8143000260DF100
:1000F0001408DDF810E03868A021002204ABCDF828
:1001000004E0CDF8008000F073FB01230222EB61D4
:10011000AA6104230822EB61AA6110232022EB616B
:10012000AA6140238022EB6131461D48AA6100F09C
:1001300049FD00200390039B711CA34205DC039B37
:100140005A1C03920398A042F9DD01230222AB61FD
:10015000EA6104230822AB61EA6110232022AB612B
:10016000EA6140238022AB610D48EA6100F02AFD7C
:100170000020039003990236A142BADC039A501C76
:1001800003900399A142F9DDB3E700BF1800001006
:10019000941100001400001040C00920FFFF0F0060
:1001A00098110000684620F007018D46F1B500F077
:1001B000B1F84F484F49884235D04F4CA14232D216
:1001C000024652F8046B0B46CD4343F8046B6519A5
:1001D000A342C5F3810526D29DB1012D0BD0022D7E
:1001E00005D0156800F108021D6001F1080352F8FE
:1001F000040B43F8040B52F8041B43F8041BA342FE
:1002000011D296465EF8047B5668D568DEF8040085
:100210009C464CF8047B5E60CCF80400DD60103333
:100220001032A342EDD335483549884234D0354C9D
:10023000A14231D2024652F8046B0B46CD4343F83B
:10024000046B6519A342C5F3810525D29DB1012D2B
:100250000BD0022D05D0156800F108021D6001F1D8
:10026000080352F8040B43F8040B52F8041B43F83C
:10027000041BA34210D294465CF8047B5668D568F0
:10028000DCF80400194641F8047B5E604860DD60DC
:1002900010331032A342EED31B491C48814221D2B5
:1002A00000220B46CC4343F8042B04198342C4F3C9
:1002B000810417D264B1012C06D0022C1CBF1A6035
:1002C00001F1080343F8042B43F8042B834209D2BD
:1002D0009E464EF8042B5A60CEF80420DA601033A4
:1002E0008342F5D3FFF7EEFEBDE8F1408546704747
:1002F000E0110000000000100C000010E0110000F0
:1003000000000010000000100C0000101C00001085
:10031000FEE700BF3649202330B4C1F8A031D1F840
:10032000A001334A10F0400FF9D0324D0124AA2029
:1003300055230321C2F80411C2F80C411146C2F83A
:100340008450C2F88C00C2F88C30C2F88040C2F8E9
:100350008C00C2F88C30D1F88830254A13F0806FB9
:10036000F9D00321AA245520C2F88010C2F88C408D
:100370001146C2F88C00D1F888301D4A13F0407F36
:10038000F9D02324C2F8A440AA2055230124C2F89E
:10039000AC001146C2F8AC30C2F8A040C2F8AC00C4
:1003A000C2F8AC30D1F8A830114A13F4806FF9D0FC
:1003B0000321AA235520C2F8A010C2F8AC30114680
:1003C000C2F8AC00D1F8A800094A10F4407FF9D077
:1003D0000949002043F23A03C2F8A801C2F8AC016F
:1003E000C2F8C410C2F8C801136030BC704700BF27
:1003F00000C00F4063000500DE87280430B5254D9E
:10040000254BD5F8C41083B041F08074C5F8C440C2
:10041000D5F8C420002042F01001C5F8C4101A68B5
:10042000044642F010051D60196821F020021A6090
:100430001D6845F0400119601A6822F080051D60B2
:10044000196841F480121A601D6825F400111960C2
:100450001A6842F480051D601968104D21F40002ED
:100460001A6000F0BBF90822012328604FF41641FE
:10047000009400F095F9022000F0B0F9084D4FF417
:100480001641286008220123009400F089F903B086
:1004900030BD00BF00C00F4000C002401800001077
:1004A0000C00001038B51F4C1F49D4F8C4301F4849
:1004B00043F40045C4F8C4500A686FF0FF0542F0E9
:1004C000FF030B60CD6100F0ABFA00F039FB184D73
:1004D0002860184800F0A4FA00F032FB2860FFF70B
:1004E0008DFFD4F8C420144942F08000C4F8C40041
:1004F0004B68002043F480024A604B6823F40002FA
:100500004A604B6843F080724A604B6823F0007287
:100510004A6000F035FA094B0949186000F03AFAD0
:10052000002038BD00C00F4040C00920002D31011F
:10053000100000100087930300C002401400001058
:10054000A0860100024B0146186800F003B800BF06
:1005500018000010436913F0200FFBD001607047B2
:1005600030B42A4A84B00DF1040C04460D46284BE1
:1005700007CAACE803009C428CF8002029D018DDA3
:10058000244B9C421BD003F580418C4214D104A91A
:100590004D19214B15F80C0CD3F8AC11820442EA2A
:1005A0000101C3F8AC11D3F8AC010240C3F8AC218F
:1005B00002E01A4884421ED004B030BC70470DF1EE
:1005C000100C6544144B15F80C2CD3F8AC11120424
:1005D000E5E704A94D19104B15F80C0CD3F8A81138
:1005E000020242EA0101C3F8A811D3F8A8010240AF
:1005F000C3F8A821E0E70DF1100C6544064B15F88F
:100600000C2CD3F8A8119201EBE700BFB411000045
:10061000000001400080094000C00F4000C00040C1
:100620002DE9F047044682B00F46002853D000F071
:1006300087FA554E554B804630689C42019000F039
:100640009C804BDD524B9C425DD003F5804294422E
:100650005FD0002302A800EB030E1EF804CC3F017C
:10066000B8FBFCF3BB422BD2D6F80090474DDFF825
:1006700020A1AC42CDF8049067D050DC454B9C42A1
:1006800035D000230DF1080E0EEB030C1CF8041CF2
:10069000012920D049082046FFF762FF3268AC42AA
:1006A00001925ED046DC3B48844226D0002302A95A
:1006B00001EB030E1EF804CCB8FBFCF3BB42D8D30D
:1006C000E268B3FBF7F342F08001E1602360E06889
:1006D00020F08002E26002B0BDE8F0872D498C4234
:1006E000B7D12D48D0F8A831C3F38113B2E72A4817
:1006F000D0F8A821C2F38113C4E7274AD2F8A81181
:10070000C1F38113D3E72448D0F8AC31C3F30143DC
:10071000A0E7214AD2F8AC11C1F381439AE75445CE
:1007200019D01E498C42ACD11B49D1F8AC31C3F36E
:100730008143A7E754451AD0184B9C42B6D1164BBB
:10074000D3F8AC01C0F38143B1E71349D1F8A83124
:10075000C3F3012396E71048D0F8AC21C2F301435C
:1007600090E70D4BD3F8A801C0F301239FE70A4A95
:10077000D2F8AC11C1F3014399E7074AD2F8A811A6
:10078000C1F3012366E700BFC01100000000014073
:100790000080094000C0004000C00F4000C0094078
:1007A00030B4092A9DF808400ED8013BDDB2053A65
:1007B000012D0ED90023072C0ED900259C18641991
:1007C000C46030BCFFF72CBF013BDDB20322012D1A
:1007D000F0D89B00072CF0D8E500EFE703289ABF7C
:1007E000024B53F820000020704700BFA411000006
:1007F0002DE9F00F099D0446282728684900A761C4
:100800000027089EC9B202302F606768F82FFCD11C
:10081000202727604FF0040C4FF008094FF0000A22
:100820004FF02808002840F39B80276817F0080F36
:10083000FBD06768083F302FF7D80FF2080B5BF842
:1008400027F000BF3B0900002B0800002B08000028
:100850002B0800002B0800002B0800002B080000CC
:100860002B0800004B0900002B0800002B0800009B
:100870002B0800002B0800002B0800002B080000AC
:100880002B080000230900002B0800002B080000A3
:100890002B0800002B0800002B0800002B0800008C
:1008A0002B080000610900002B0800002B08000045
:1008B0002B0800002B0800002B0800002B0800006C
:1008C0002B080000090900002B0800002B0800007D
:1008D0002B0800002B0800002B0800002B0800004C
:1008E0002B080000610900002B0800002B08000005
:1008F0002B0800002B0800002B0800002B0800002C
:100900002B080000610900001F68A160012FC4F8D6
:1009100000C0C4F818902BDD013F12F8011B1F60C6
:1009200080E71F68A160012FC4F800A0C4F81890E8
:10093000F2DC013816F8011B74E7A160C4F800C0AE
:10094000C4F8188012F8011B6CE71F68A160013F12
:10095000C4F800C0C4F8188012F8011B1F6061E7DA
:100960001422082322600020A361BDE8F00F704725
:10097000296801380131296016F8011B52E700BFD0
:1009800002289ABF024B53F820000020704700BF96
:10099000C811000030B5044683B00D4618B300F00E
:1009A000CFF81B490B6801931A4B9C4224D003F5E6
:1009B0008822944226D0184B9C4216D0002302AACB
:1009C000D11811F804CC6C23B0FBFCFEBEFBF5F58E
:1009D0006D08032D98BF042540222820A3612561BE
:1009E00065612260A06103B030BD03F5602CDCF8C6
:1009F000A831C3F38133E2E7084AD2F8AC11C1F35E
:100A00008113DCE70549D1F8AC31C3F30153D6E7D4
:100A1000C411000000C0054000C0014000C00F40EC
:100A2000F0B4404D3F4CD5F80C31D4F80C1113F014
:100A3000030F08BF3C4B3B4E01F003070CBF1A6885
:100A400042F21072D6F80C51012F08BF374F05F053
:100A5000030308BF3A68022B08BF354B314908BF72
:100A60001A68344BB3FBF0F4601EC1F80401500067
:100A7000012218E0B4FBF0F1CF1F0132B7F5FC7F83
:100A8000144622D9B5FBF0F1CD1F0132B5F5FC7F3C
:100A90001BD9B6FBF0F1CD1FA21CB5F5FC7F14D914
:100AA000E21C212A3BD02349234F244E5C18B3FB80
:100AB000F0F1DD199E19CF1F03F18E4303F5060CEB
:100AC000B7F5FC7F0CF50C43D4D8541E154B22040B
:100AD00001398918AA2455200122C3F88410C3F8CB
:100AE0008C401946C3F88C00C3F88020C3F88C40B2
:100AF000C3F88C00D1F888000A4A10F0806FF9D052
:100B00000321AA205523C2F88010C2F88C00114698
:100B1000C2F88C30D1F8882012F0407FFAD0F0BCB7
:100B2000704700BF00C00F4004000010000000101C
:100B30000800001000A3E1110046C32300E9A4351A
:100B40001C4A30B4D2F88450D2F88440D2F8041150
:100B5000D2F80C3113F0030F04BF174B1868154B74
:100B6000D3F80C2102F0030C124ABCF1010FD2F8A9
:100B70000C2108BF114B02F0030C08BF1868BCF130
:100B8000020F04BF0E4B18680A4BD3F8802012F0F6
:100B9000020F0CD0AA04930C5A1C5300C4F3074450
:100BA0004A1C00FB03F004FB0221B0FBF1F030BC57
:100BB000704700BF00C00F4004000010000000108C
:100BC000080000100FB42DE9F04784B00CAB53F8C7
:100BD000045BDFF8FC803D4F00240393287840B18C
:100BE00025280CD00135FFF7ADFC2878013400280A
:100BF000F6D1204604B0BDE8F04704B070476878ED
:100C0000013525285DD02538532855D8DFE810F068
:100C10009C025400540054005400540054005400EA
:100C20005400540054005400540054005400540024
:100C30005400540054005400540054005400540014
:100C40005400540054005400540054005400540004
:100C500054005400540054005400540054005400F4
:100C600054005400540054005400540054005400E4
:100C70005400540054005C015400540054005400CB
:100C800054005400540054005400540054016200B5
:100C900054005400540054005400540054005400B4
:100CA00054005400540054005400540054005400A4
:100CB000540054005400FB0103980135021D0392B7
:100CC0008CE7FFF73FFC0135013487E7676666660E
:100CD000D4110000039BEC46D3F8009098E807007D
:100CE000ACE803000020043381456E4603938CF882
:100CF00000208DF80900C0F22C82B9F1000F40F3FA
:100D0000D98087FB09204FEAE971C1EBA00303EB0F
:100D1000830EA9EB4E0A0AF130098DF80090002BE2
:100D200000F0208287FB03C9DA17C2EBA90202EBAD
:100D3000820CA3EB4C0330338DF80130002A00F015
:100D40000E8287FB023ED017C0EBAE0303EB830A93
:100D5000A2EB4A0130318DF80210002B00F0048222
:100D600087FB03C9DA17C2EBA90202EB820CA3EBE3
:100D70004C0330338DF80330002A00F0FB8187FBF1
:100D8000023ED017C0EBAE0303EB830AA2EB4A018D
:100D900030318DF80410002B00F0E98187FB03C986
:100DA000DA17C2EBA90202EB820CA3EB4C0330333F
:100DB0008DF80530002A00F0E08187FB023ED01755
:100DC000C0EBAE0303EB830AA2EB4A0130318DF88E
:100DD0000610002B00F0D78187FB03C9DA17C2EB9E
:100DE000A90202EB820CA3EB4C0330338DF80730E1
:100DF000002A00F0C58187FB023ED017C0EBAE038E
:100E000003EB830AA2EB4A0130318DF80810002B66
:100E100000F0BC8187FB03C9D817C0EBA90202EB25
:100E2000820CA3EB4C0330338DF809304FF0090AE4
:100E300016F80A00FFF786FBBAF1000F0AF0030369
:100E40000AF1FF3936DDD3B1012B0DD0022B05D0CD
:100E500016F80900FFF776FB09F1FF3916F80900CB
:100E6000FFF770FB09F1FF3916F8090009F1FF39A6
:100E7000FFF768FB09F1010CBCF1000F1ADD16F851
:100E8000090009F1FF3AFFF75DFB16F80A00A9F126
:100E9000020AFFF757FB16F80A00FFF753FBA9F108
:100EA0000303F05CA9F10409FFF74CFB09F1010110
:100EB0000029E4DC013591E6039A0135111D107813
:100EC0000391FFF73FFB89E603996E460A68081D08
:100ED00002F00F03092B88BF0733039098E8030043
:100EE00086E80300111101F00F003033092888BF94
:100EF00007300A118DF8003002F00F033030092B53
:100F000088BF073311118DF8010001F00F00092887
:100F100088BF0730091101F00F023030092A88BF5D
:100F2000073203F130090B118DF8030003F00F00B5
:100F3000092888BF07301B1102F1300C03F00F02A3
:100F4000092A00F1300188BF0732C3F303103032A1
:100F5000092888BF073030308DF802908DF804C022
:100F60008DF805108DF806208DF80700082300E0A5
:100F70004B4603F1FF3916F809003028F8D0002B52
:100F800098DDFFF7DFFAB9F1000F09F0030309F16B
:100F9000FF3A8FDDD3B1012B0DD0022B05D016F80F
:100FA0000A00FFF7CFFA0AF1FF3A16F80A00FFF736
:100FB000C9FA0AF1FF3A16F80A000AF1FF3AFFF7F8
:100FC000C1FA0AF1010100297FF774AF16F80A008F
:100FD0000AF1FF39FFF7B6FA16F80900AAF102097B
:100FE000FFF7B0FA16F80900FFF7ACFAAAF103030D
:100FF000F05CAAF1040AFFF7A5FA0AF1010CBCF1B2
:10100000000FE3DC56E703996E460A68081D02F0FC
:101010000F03092B88BF2733039098E8030086E865
:101020000300111101F00F003033092888BF273069
:101030000A118DF8003002F00F033030092B88BF01
:10104000273311118DF8010001F00F00092888BF26
:101050002730091101F00F023030092A88BF2732EA
:1010600003F1300C0B118DF8030003F00F00092879
:1010700088BF27301B1102F1300903F00F02092A43
:1010800088BF27328DF802C000F1300CC3F3031083
:101090003032092888BF273030308DF804908DF821
:1010A00005C08DF806208DF80700082300E04B46A8
:1010B00003F1FF3916F809003028F8D0002B7FF72C
:1010C000F9AEFFF73FFAB9F1000F09F0030309F198
:1010D000FF3A7FF7EFAED3B1012B0DD0022B05D035
:1010E00016F80A00FFF72EFA0AF1FF3A16F80A007E
:1010F000FFF728FA0AF1FF3A16F80A000AF1FF3A58
:10110000FFF720FA0AF10103002B7FF7D3AE16F8A0
:101110000A000AF1FF39FFF715FA16F80900AAF1DB
:101120000209FFF70FFA16F80900FFF70BFAAAF108
:101130000303F05CAAF1040AFFF704FA0AF1010CB8
:10114000BCF1000FE3DCB5E625200135FFF7FAF925
:1011500044E52D20C9F10009FFF7F4F9CDE54FF082
:10116000010A65E69A4663E64FF0020A60E64FF030
:10117000040A5DE64FF0030A5AE64FF0050A57E607
:101180004FF0070A54E64FF0060A51E64FF0080AFE
:101190004EE600BF010500007465737420256420CD
:1011A0000A0D000000C0004000000140008009401E
:1011B00000C009400101020200000000030000001D
:1011C000040102080401020800C0014000C00540FB
:1011D00000000A40202020202020202000000000C5
:0C11E000001BB70000093D00008000006B
:00000001FF
